:020000040000FA
:020000000528D1
:0800080005280730990083165A
:100010009F01F83085008330810083120514851418
:1000200005150511851910288320851D1428051034
:1000300005150000000000000000000000000000A6
:1000400000000000000000000000000000000000B0
:1000500000000000000000000000000000000000A0
:10006000000005110000000000000000000000007A
:100070000000000000000000000000000000000080
:1000800000000000000000000000000000008519D2
:1000900018288320851D4928051485100515523020
:1000A000A400A40B5128051100000000000000006E
:1000B0005130A400A40B5A2885194E288320851D91
:1000C0005E2805100515FA30A400000000000000AD
:1000D0000000000000000000A40B65280511F930A5
:1000E000A40000000000000000000000000000006C
:1000F000A40B7128000000000000851962288320ED
:10010000851D7F280E28A501A401A40B8528A50B19
:10011000852808000528052805280528052805281C
:100120000528052805280528052805280528052867
:100130000528052805280528052805280528052857
:100140000528052805280528052805280528052847
:100150000528052805280528052805280528052837
:02400E00C23FAF
:00000001FF
